:10000000170500001305C515970500009385A51574
:1000100093081008730000009705000093852515CC
:10002000730000009308500873000000630105127C
:10003000930860087300000093081008170500007B
:1000400013050513970500009385651373000000E1
:100050000F000001970500009385951273000000C2
:100060000F000001970500009385651173000000E3
:100070000F000001970500009385951073000000A4
:100080000F000001970500009385650F73000000C5
:100090000F000001970500009385950E7300000086
:1000A0000F000001970500009385650D73000000A7
:1000B0000F000001970500009385950C7300000068
:1000C0000F000001170500001305F50A9705000051
:1000D0009385E50A730000000F00000197050000FA
:1000E0009385150A730000000F00000197050000BA
:1000F0009385E508730000000F00000197050000DC
:1001000093851508730000000F000001970500009B
:100110009385E506730000000F00000197050000BD
:1001200093851506730000000F000001970500007D
:100130009385E504730000000F000001970500009F
:1001400093851504730000000F000001E1BD73D01A
:1001500000800F00000173500080E9B574696D657F
:1001600072006C6F6F705F6F6E0031006C69676852
:100170007431006C696768743200313400300000FB
:00000001FF
